:100000006528920024088400F030A1050830930090
:1000100003100318A10A1A20920C930B0928000060
:10002000971A210C1A20632003141A201B088F0032
:100030001A083F288413971F292800082204171F35
:1000400022068000841700082204031C2206800078
:10005000342800082204031C2206171B22068000F5
:10006000841722098005342817081F39FF3E8D00A8
:100070001608F53E03188D0A00004C288F018E00EB
:10008000FF308E07031C8F07031C602803308D0090
:10009000DF304C2040288D01E83E8C008D09FC307B
:1000A000031C55288C07031852288C0764008D0FF9
:1000B00052280C185B288C1C5F2800005F28080061
:1000C0008313031383126400080083161030850025
:1000D000013086008113831279280530A40008308E
:1000E000A2005430960097019A019B013130012003
:1000F000080085018601861083168610053083125C
:100100003E20640006187B2886148316861083120E
:100110006D2001308F00F4303F207B2863008E2853
:02400E00F53F7C
:00000001FF
